:100000000C94E5020C9451290C941D030C941D03CF
:100010000C941D030C941D030C941D030C941D03E0
:100020000C941D030C941D030C941C200C94581F5D
:100030000C94D7190C941D030C941D030C941D03F0
:100040000C941D030C941D030C941D030C941D03B0
:100050000C941D030C948A190C941D030C941D031D
:100060000C941D030C941D030C941D030C941D0390
:100070000C941D030C941D030C941D030C941D0380
:100080000C941D030C941D030C941D030C941D0370
:100090000C941D030C941D030C941D030C941D0360
:1000A0000C941D030C941D030C941D037F077F0704
:1000B000B107B1072308CB09CB09CB093F081D09BC
:1000C0002E092E09711D981D301F981D301FE01D2F
:1000D000031E301FF21E051F00047F3F1F643214F1
:1000E000643214783C1E1E140A0522232526282972
:1000F0002A2C2D2F3032333536383A3B3D3E4042A4
:10010000434547494A4C4E5051535557595A5C5EE6
:100110006062646668696B6D6F71737577797B7DFA
:100120007F81838587898A8C8E90929496989A9CF9
:100130009E9FA1A3A5A7A8AAACAEAFB1B3B4B6B811
:10014000B9BBBCBEBFC1C2C3C5C6C7C9CACBCCCD73
:10015000CED0D1D2D2D3D4D5D6D7D7D8D9D9DADA4E
:10016000DBDBDBDCDCDCDCDCDDDDDDDDDCDCDCDCCE
:10017000DCDBDBDBDADAD9D9D8D7D7D6D5D4D3D202
:10018000D2D1D0CECDCCCBCAC9C7C6C5C3C2C1BFE0
:10019000BEBCBBB9B8B6B4B3B1AFAEACAAA8A7A544
:1001A000A3A19F9E9C9A98969492908E8C8A898700
:1001B0008583817F7D7B79777573716F6D6B6968DE
:1001C000666462605E5C5A5957555351504E4C4AB2
:1001D0004947454342403E3D3B3A3836353332305D
:1001E0002F2D2C2A29282625232205010980A1014B
:1001F000850319012AB700150126B700950175106E
:100200008100C0050C0901A101850419012AA00281
:10021000150126A002950175108100C0050109068F
:10022000A101050719E029E71500250195087501C9
:1002300081029501750881010507190029FF150044
:1002400026FF009506750881000508190129059506
:100250000575019102950175039101C009023B00EA
:10026000020100A0FA0904000001030101000921B4
:100270001101000122400007058103080001090463
:1002800001000103000000092111010001223200D8
:10029000070582032000011201000200000008107F
:1002A000CB561200030102000126034B00650065D6
:1002B00000620069006F002000490072006900734D
:1002C0000020005200650076002E00200033000060
:1002D000000E034B0065006500620069006F0000BE
:1002E000000403090429001E001F00200021002231
:1002F000002B0014001A00080015001700E000048D
:10030000001600070009000A00E1001D001B00069E
:100310000019000500000000004A00E300A85D2865
:10032000002A00270026002500240023004C00138B
:100330000012000C0018001C00340033000F000EE7
:10034000000D000B00E500380037003600100011EA
:1003500000000000004D00E600A95D2C0035021EE3
:10036000021F02200221022202005C1E001F002048
:1003700000210022004C00010050004F0052002FCD
:1003800000C15C01000100010051002F02000000CB
:10039000002602010001004C002A00270226022547
:1003A0000224022302010027002600250024002346
:1003B0000031022E025E005D005C00300001002D65
:1003C000005B005A00590030020000000027026262
:1003D0000001004C0045003A003B003C003D003E5F
:1003E00000C35C1E021F02200221022202C45CAC78
:1003F00000AB00A9004B002D02A800AD00AE00AA82
:10040000004E002D00000000002602010001000146
:1004100000440043004200410040003F000100272B
:100420000226022502240223023100CA5CC85CC6EF
:100430005C4A002E000100CB5CC95CC75C4D002EFD
:1004400002000000000100010001000100010001A4
:100450000001000100010001000100010001000194
:100460000001000100010001000100010001000184
:100470000001000100010001000100010000000076
:100480000001000100010001000100010001000164
:100490000001000100010001000100010001000154
:1004A0000001000100010001000100010001000144
:1004B0000001000100010001000000000001000136
:1004C000000100010000010101010101010101021F
:1004D00002020202020202020303030303030303F4
:1004E00004040404040404050505050506060606BF
:1004F00006070707070708080808090909090A0A7B
:100500000A0B0B0B0C0C0C0D0D0D0E0E0E0F0F0F1E
:1005100010101111111212131314141515161617A9
:1005200017181819191A1A1B1B1C1D1D1E1E1F2017
:1005300020212222232424252626272829292A2B64
:100540002C2D2D2E2F303132323334353637383989
:100550003A3B3C3D3E3F4041424344454647484983
:100560004A4C4D4E4F50515354555658595A5B5D55
:100570005E5F616264656668696B6C6D6F707273F3
:100580007577787A7B7D7E8082838587888A8C8E5A
:100590008F91939596989A9C9EA0A2A3A5A7A9AB8C
:1005A000ADAFB1B3B5B7BABCBEC0C2C4C6C9CBCD7E
:1005B000CFD1D4D6D8DBDDDFE2E4E7E9EBEEF0F330
:1005C000F5F8FAFDFFFFAA7F554011241FBECFEFBB
:1005D000DAE0DEBFCDBF04B603FE18C0809115037C
:1005E00090911603A0911703B09118038730904B98
:1005F000A740B04B59F410921503109216031092B5
:10060000170310921803E0E0F8E3099511E0A0E069
:10061000B1E0E4E1F7E502C005900D92AC3CB10712
:10062000D9F723E0ACECB1E001C01D92A531B207CF
:10063000E1F70E941A0C0C94882B0C9400001F9375
:10064000CF93DF93CDB7DEB767970FB6F894DEBFD1
:100650000FBECDBF4B8B5C8B6D8B7E8B8F8B6111F7
:100660001092140386E09E01235F3F4FD901E82FCB
:100670001D92EA95E9F795E0FE017396D901019084
:100680000D929A95E1F79C894E895F897B897D87D8
:100690009E876F87598B488BF901DE011796019071
:1006A0000D928A95E1F7CE0107960E9446228111AC
:1006B0003EC086E0FE013796DE01119601900D9254
:1006C0008A95E1F7FF81E8856A857B85611571056B
:1006D00031F0EF3F31F481E0FF3F19F403C081E0D6
:1006E00001C080E080FD23C02091D90230E0C90123
:1006F00001968770992740910A0350E08417950767
:1007000079F1F983EA837D836C8396E0929FD0012F
:10071000939FB00D1124A652BD4FFE01319601905A
:100720000D929A95E1F78093D9020E943B2116E041
:1007300080910A039091D9028917F9F0189FC0019E
:10074000112486529D4F0E9446228823B1F0809149
:100750000A0390E001968770992780930A03E8CFF7
:100760000E94D4241092D90210920A03E3EDF2E021
:1007700086E0DF011D928A95E9F767960FB6F89437
:10078000DEBF0FBECDBFDF91CF911F9108958111C4
:1007900006C0662311F089EA09C08AEA07C08130E1
:1007A00039F4662311F08EE401C08BE40E94F0243A
:1007B00080E008958F929F92AF92BF92CF92DF9286
:1007C000EF92FF920F931F93CF93DF93CDB7DEB7D6
:1007D0002A970FB6F894DEBF0FBECDBFFC01008193
:1007E000D18083819481892B39F01FEFD11206C00B
:1007F00091E00F3F19F403C091E001C090E090FD3B
:10080000F6C67F0185E0DE01169601900D928A956D
:10081000E1F7F70122818E819F81222349F00E9416
:10082000B121182F682F8E819F810E94142403C04C
:100830000E94E723182F2CE3129FF001112436E0C9
:10084000D39EE00DF11D1124E00FF11DEE0FFF1FEF
:10085000EB51FD4F05911491F7018281083AFDE5B6
:100860001F07F1F028F4073A3DE5130751F034C0B3
:10087000093A9DE51907F1F00A3AEDE51E0711F175
:100880002BC0882309F4DBC561E083E090E00E947F
:10089000862A61E070E080E090E00E94CA24CFC523
:1008A000882311F081E009C081E00E944A240E945F
:1008B000411CC5C5882321F082E00E94A924F7CFFE
:1008C00082E0F3CF882321F083E00E94A924B7C5FA
:1008D00083E00E944A24B3C5882309F482C00E3BFA
:1008E000FCE51F07E1F058F40C3B3CE5130799F0D9
:1008F0000D3B9CE5190709F074C080E00DC0003C79
:10090000ECE51E0709F45DC008F442C0013C2CE58B
:100910001207A9F066C085E00E94A51B90C58091D2
:100920007602982F96959695969561F1915E990F1E
:10093000990F990F8770892B8093760217C0809149
:100940007602282F2695269526952F5F2F71922FB8
:10095000990F990F990F8770892B80937602263013
:1009600018F087708093760280917602887F91E0FC
:1009700009F490E08091760290FB80F980937602F2
:100980000E94A01B8091760286958695869523C04D
:1009900020917602822F869586958695482F50E085
:1009A0004530510554F48F5F982F990F990F990F87
:1009B000822F8770892B80937602809176028160E6
:1009C000DDCF8091760280FF09C08E7F8093760212
:1009D0000E94A01B80E00E94ED1A31C50E94C21B3C
:1009E0002EC5043F2CE5120799F406E221EE40EEF5
:1009F00064EF7CE509C0083DFCE51F0711F506E240
:100A000021EE41EE68ED7CE5C7010E94631A17C52F
:100A1000053F3CE5130708F05CC1093D9CE519075B
:100A200031F407E225EE45EE69ED7CE5EDCF0A3DB8
:100A3000ECE51E0701F708E221E045EE6AED7CE5F2
:100A4000E3CF882309F47AC11092790204303DE59E
:100A5000130758F40B3F8CE5180780F4C801825047
:100A60009C45449708F054C109C002369DE519071A
:100A700029F0063AEDE51E0709F04AC10E9400136D
:100A800090930602809305020131FCE51F0709F4EB
:100A9000C6C008F042C009303CE5130709F49BC00A
:100AA00000F505309CE5190709F485C078F403309A
:100AB000FCE51F0709F478C008F07AC002301C4535
:100AC00009F0F7C0809105028160F1C007308CE524
:100AD000180709F478C008F07AC080910502806197
:100AE000E6C00D30ECE51E0709F487C058F40B3062
:100AF0002CE5120709F479C008F07BC0809105024B
:100B000088606FC00F308CE5180709F480C008F0CA
:100B100082C080910502877FCAC00E3FECE51E07A8
:100B200009F471C000F505312CE5120709F485C000
:100B300068F403318CE5180709F475C008F095C016
:100B40000E94D424809105028F77B1C00C3FECE560
:100B50001E07A9F108F054C00B3F1C4509F0A9C0BD
:100B60008091060240C002303DE5130709F489C0B8
:100B700058F401159DE5190709F45AC008F069C039
:100B80008091060282602FC00236FDE51F0709F43E
:100B90007EC0063A2DE5120709F483C003301D45D7
:100BA00009F087C060E06EC08091050282607FC05E
:100BB0008091050216C080910502886078C08091FE
:100BC000060282604FC080910502806270C08091F1
:100BD000050280646CC00E94D42480910502806864
:100BE00066C0846064C081603DC0809105028E7FD4
:100BF0005EC0809105028D7F5AC08091050216C0AB
:100C00008091060218C0809106028D7F2BC08091D2
:100C100005028F7E4CC0809105028F7D48C0809177
:100C200005028F7B44C080910502877F8B7F3FC088
:100C3000809106028D7F8E7F15C08091050282FB18
:100C4000222720F991E0922790FB82F990FB83F90B
:100C50002EC080910602982F909591708E7F892BDF
:100C600090FB81F98093060224C00E94D4248091D5
:100C7000050287FB222720F991E0922790FB87F954
:100C800016C061E08EE090E00E94862A12C080913A
:100C9000050284FB222720F991E0922790FB84F93A
:100CA00006C080910502982F909590FB80F9809363
:100CB0000502609105021091060284E090E00E9416
:100CC000862A612F82E290E00E94862A0E94D42424
:100CD000B6C3063F2CE5120731F406E221EE42EEE0
:100CE00066EF7CE591CE063F3CE5130730F407E262
:100CF00025EE44EE65EF7CE587CE073F9CE51907BE
:100D000009F09FCE07E225EE46EE67EF7CE57CCE4C
:100D10000631ECE51E0721F5809127028A7A91E0E1
:100D200009F490E09093CE01882311F065E301C0AF
:100D300069E283EA92E00E940D1A0FC00631FCE5D9
:100D40001F0709F064C08091CE01882309F49AC37B
:100D500065E383EA92E00E94001A0E94F3206FC3C9
:100D60000B35FDE51F0709F44CC058F401153CE5AF
:100D70001307C1F00F3D1C4509F065C00E94111317
:100D80005EC30C359DE5190709F43DC00D351D45C1
:100D900009F059C08091060282FB882780F991E012
:100DA000892732C00E94D424FFEF04E31CE0F150F5
:100DB00000401040E1F700C0000081E08093E000B7
:100DC00080E28093D8001092C9008FE19EE40197E1
:100DD000F1F700C0000087E090EBDC018093150381
:100DE00090931603A0931703B09318039CE088E137
:100DF0000FB6F894A895809360000FBE90936000A2
:100E0000FFCF81E001C080E00E948C241CC0809153
:100E1000270282720D3C9CE5190709F4CAC308F049
:100E2000F7C2073CFCE51F0709F4AFC308F03AC35B
:100E3000043C3CE5130709F49EC308F025C3033CBA
:100E40001C4509F46FC3F70182810081D18088239A
:100E500059F0802F9D2D0E94B121182F682F802FCF
:100E60009D2D0E94142405C0802F9D2D0E94E723F4
:100E7000182F2CE3129FF001112436E0D39EE00DD1
:100E8000F11D1124E00FF11DEE0FFF1FEB51FD4F7F
:100E9000859194910E9475118C01982EF701D28052
:100EA000A580A2943FE0A32280910B038770B9F044
:100EB000DD20A9F0812F807F803421F080E2800F37
:100EC000883068F08091060282FD09C082E00E94AD
:100ED0006F2480910B038770CC24C3948111C12CA3
:100EE000B12EB2949FE0B9228B2D90E08C30910509
:100EF00008F051C2FC01EA5AFF4F0C94222B812FBB
:100F0000807F1F70882311F01295107FDD20B9F0CB
:100F1000112309F42DC280E2800F883010F0911067
:100F200006C080912702182B1093270205C08091DC
:100F30001403182B109314030E94F32019C2802F5E
:100F40000E94BD27112309F426C2005E083078F103
:100F5000992069F1109580911403182310931403BC
:100F600029C0812F807F1F70803211F01295107F71
:100F7000992021F0F1E09F16D9F149C08091060235
:100F800082FF1BC0DD2069F0112339F08091270218
:100F9000182B109327020E94F32080E00E9414284F
:100FA000FAC180E00E94BD27112309F4F4C1812F0A
:100FB0000E9498130E94F320EEC1DD2081F0809101
:100FC0002802AA2051F001E0A01207C0182B181720
:100FD00009F4E1C110932802DEC1812B10C0AA20C0
:100FE00021F021E0A21609F4D6C10E94921327C075
:100FF000DD2041F035E03A1508F4CDC1812F0E9483
:10100000E624C9C184E08A1508F4C5C118C0DD20F2
:1010100049F0AA2099F3F701858180FFA9C18F705B
:101020008583ECCFAA2059F0093309F0B1C1FFEF55
:1010300017EE23E0F15010402040E1F7A7C1812FC7
:101040000E94DF24A8C1812F86958695837019F0B0
:10105000813059F0A0C1DD2019F0C801937002C0A1
:1010600080E090E00E943D1A9CC1DD2019F0C8018B
:10107000937002C080E090E00E94271A92C1812FF5
:10108000837009F069C0D1108AC1902F929596950E
:101090009770990F990F802F8F70882E912CA12C0B
:1010A000B12C092E04C0880C991CAA1CBB1C0A94E4
:1010B000D2F704FF12C04FE050E060E070E004C0DF
:1010C000440F551F661F771F9A95D2F7DB01CA019F
:1010D00080959095A095B09503C080E090E0DC01EC
:1010E00016951695412F4370423019F1C8F40091BE
:1010F000290210912A0220912B0230912C024130BA
:1011000059F088299929AA29BB29BC01CD0160235E
:101110007123822393230AC0802A912AA22AB32A08
:10112000BC01CD01682979298A299B290E94CA24FA
:1011300036C188299929AA29BB2900912902109131
:101140002A0220912B0230912C02BC01CD01602794
:10115000712782279327EACFDD2019F0812F817034
:1011600001C08695882309F41AC1902F929596950F
:101170009770990F990F802F8F70882E912CA12C2A
:10118000B12C092E04C0880C991CAA1CBB1C0A9403
:10119000D2F704FF12C04FE050E060E070E004C0FE
:1011A000440F551F661F771F9A95D2F7DB01CA01BE
:1011B00080959095A095B09503C080E090E0DC010B
:1011C00016951695412F43704230D9F068F500917D
:1011D0009F021091A0022091A1023091A202413001
:1011E00059F088299929AA29BB29BC01CD0160237E
:1011F0007123822393231EC0802A912AA22AB32A14
:1012000013C088299929AA29BB2900919F0210910E
:10121000A0022091A1023091A202BC01CD01602761
:1012200071278227932706C0BC01CD01682979293F
:101230008A299B290E944024B2C01F70DD2039F00A
:10124000812F0E94A924802F0E94E624A8C0802F0D
:101250000E94DF24812F0E944A24A1C0802F32EFF8
:10126000931609F443C0391538F090EF991659F0E8
:10127000E1EF9E16B1F177C0F3EF9F16F1F124EF85
:10128000921659F170C0DD2019F134E03A1508F4D6
:1012900082C01F7181E090E0A0E0B0E0AC01BD0130
:1012A00004C0440F551F661F771F1A95D2F780910F
:1012B0009F029091A002A091A102B091A2028A0186
:1012C0009B01082719272A273B27C901B80129C0F4
:1012D00025E02A1508F45FC0DCCF8091060282FF6A
:1012E00023C0DD2029F0812F8F7130C0DD20D9F39C
:1012F000812F8F710E944A244EC0DD2079F01F712A
:1013000081E090E0A0E0B0E0BC01CD0104C0660F38
:10131000771F881F991F1A95D2F703C060E070E00D
:10132000CB010E94402437C0DD2099F01F71812F2E
:101330000E94A9248091060282FD07C038E0139F15
:10134000C0011124836080930B03812F0E94A92484
:1013500022C081E00E946F2481E08A15E0F482E0DF
:101360000E946F2418C0DD2029F0AA2009F4BBCF09
:10137000802F14CEAA2009F4BBCF893349F49FEF04
:10138000E7EEF3E09150E040F040E1F700C00000EC
:10139000802F0E94BD2788EF8B0D843010F40E94AF
:1013A000531ACC20A9F080910B0380FD11C0F701E6
:1013B00012828595859585950E94A924C7010E9472
:1013C000DA0380910B038595859585950E944A24C3
:1013D00085E0F701DE01119601900D928A95E1F703
:1013E00089819A810E94E7239A810CE3809FF00112
:1013F000112416E0919FE00DF11D11248981E80F61
:10140000F11DEE0FFF1FEB51FD4F85919491EFC041
:10141000023D8CE5180709F4DBC008F465C0053D02
:101420008CE5180709F4DAC008F471C0063D2CE514
:10143000120709F4D8C00E351D4509F004CD80917E
:101440000B03877009F4D3C0F7018281882309F464
:10145000CEC08091060282FDCAC082E02A960FB6F5
:10146000F894DEBF0FBECDBFDF91CF911F910F91DA
:10147000FF90EF90DF90CF90BF90AF909F908F90B4
:101480000C946F2469E265CC053CFCE51F0709F468
:1014900077C0063C1C4509F0D6CC45E557E26EE521
:1014A00077E28BC00A3C3CE5130709F478C070F47E
:1014B000083CECE51E0709F46DC0093C1C4509F029
:1014C000C2CC49E457E26DE377E277C00B3C2CE5F0
:1014D000120709F469C00C3C1C4509F0B4CC4AE978
:1014E00055E26BEA75E269C00F3CECE51E0709F4B2
:1014F00069C008F465C0003D2CE5120709F465C019
:10150000013D1C4509F09FCC6EE089E069C0033DB8
:10151000ECE51E0709F45FC0043D1C4509F093CCBF
:1015200088E162C08091710280FF20C08E7F80932D
:1015300071026091710270917202809173029091B8
:1015400074020E9488250E941F1C809149028160BC
:10155000809349028FEF90E7E2E081509040E040B5
:10156000E1F700C000000E940E2569CF81608093E2
:101570007102869539C04AEA57E263EB77E21DC0F3
:1015800043EB57E26AEA77E218C04EE557E265E5B9
:1015900077E213C04DE357E269E477E20EC045E21B
:1015A00057E261E377E209C041E357E265E277E29F
:1015B00004C04BEA55E26AE975E20E94191C3FCF6C
:1015C00081E012C065E082E00BC068E086E008C000
:1015D00064E18FE005C067E185E102C062E289E174
:1015E0000E94081C2CCF83E20E94A72728CF2A96AE
:1015F0000FB6F894DEBF0FBECDBFDF91CF911F9124
:101600000F91FF90EF90DF90CF90BF90AF909F90A1
:101610008F9008950F931F93CF93DF93CDB7DEB7CD
:1016200028970FB6F894DEBF0FBECDBF85E0E1E787
:10163000F2E0DE01119601900D928A95E1F780911A
:10164000470290914802A09149028E839F83A88708
:1016500041E08885811101C040E008E010E09E0172
:101660002F5F3F4F60EF71E086E00E94D20F811143
:101670001092490228960FB6F894DEBF0FBECDBF78
:10168000DF91CF911F910F9108950F931F93CF93E7
:10169000DF931F92CDB7DEB78091760280FF04C042
:1016A00086958695869501C080E0898341E090917A
:1016B000DF01981301C040E001E010E09E012F5FC0
:1016C0003F4F6CEE71E085E00E94D20F0F90DF91EA
:1016D000CF911F910F910895CF93DF9300D000D049
:1016E000CDB7DEB74091E8015091E9016091EA0180
:1016F0007091EB012FB7F894809181029091820252
:10170000A0918302B09184022FBF841B950BA60B7E
:10171000B70B84369105A105B10570F10E945111F6
:10172000DC01CB010296A11DB11D89839A83AB8395
:10173000BC8380912101909122018D529E4F409156
:10174000200150E04530510510F044E050E0BE016A
:101750006F5F7F4F0E947F2B84E090E00E94F7290B
:10176000882359F00E94BF196093E8017093E90142
:101770008093EA019093EB0181E00F900F900F901E
:101780000F90DF91CF910895CF92DF92EF92FF9269
:101790000F931F93CF93DF931F92CDB7DEB7EE2445
:1017A000E394F12C0AED11E09E012F5F3F4F4FECC7
:1017B00051E063E082E00E943010C82E882379F166
:1017C000D09008028D2D90E09C012F5D3D4F790156
:1017D0001981F9018081181B012F80E010165CF43B
:1017E0000150F70180818F5F808360E08D2D0E9422
:1017F000C70381E0F3CF912F17FD90E0191B112350
:1018000059F01F5FF70180818150808361E08D2D49
:101810000E94C70381E0F3CF81110E94FE128C2D3C
:101820000F90DF91CF911F910F91FF90EF90DF907C
:10183000CF900895CF93DF93CDB7DEB72A970FB639
:10184000F894DEBF0FBECDBF84B7877F84BF0FB6CD
:10185000F894A89580916000886180936000109250
:1018600060000FBE90E080E80FB6F89480936100AE
:10187000909361000FBE85B7806885BF85B780688B
:1018800085BF8DE89FE09093CD018093CC010E94AD
:101890009C1F0E94BB1F8091E20084608093E20045
:1018A0007894809195028823A1F01091E9001F702F
:1018B0009091EC00892F817090FD80E8182B109298
:1018C000E9008091E80083FD0E948B1C1F7010933B
:1018D000E90082E084BD93E095BD9AEF97BD8093C7
:1018E0006E001092F5011092F6011092F70110921D
:1018F000F801809888988FB1817080933801809129
:101900003801882321F01092530186E003C086E05D
:1019100080935301809354010E94171181110E94FA
:101920000B298091380180913801811102C095E026
:1019300001C090E09093040285E0891B809303022C
:101940000BE511E060E6E62E61E0F62ED8018D9100
:101950008D018F3F11F00E943A11E016F106B1F7A8
:1019600000E611E056E6E52E51E0F52EF8018191F2
:101970008F018F3F11F00E943A11E016F106B1F786
:101980008AE0E9E0F2E0DF01282F1D922A95E9F7CD
:10199000E9EFF1E0DF011D928A95E9F780E090E040
:1019A0000E94802A893E9E4F11F00E94111382E00E
:1019B00090E00E94722A809313020E940013909379
:1019C00006028093050283E090E00E94722A682F4D
:1019D00070E080E090E00E94CA24269A2E9882E26D
:1019E0008093800089E1809381008FEF9FEF909337
:1019F0008700809386000E94DA1B0E94DA1B809188
:101A0000070281113BC080E090E00E94802A893E5D
:101A10009E4F21F00E9411130E94BC2588E090E0A7
:101A20000E947A2A6093710270937202809373020B
:101A300090937402809149028360809349026E7F83
:101A400071F40E94BC2588E090E00E947A2A60939D
:101A500071027093720280937302909374020E94D9
:101A600075250E941F1C8091710280FF04C060E0F8
:101A700086950E94672781E08093070225982D9A1A
:101A800027982F9A8FE891E00197F1F700C00000A6
:101A900083B185FB882780F923B130E0220F232F03
:101AA000221F330B232B11F490E001C092E0892B0D
:101AB000809325029091380181E098279093240229
:101AC000891B809308020E941711811102C00E9495
:101AD0000E2989E391E090937D0280937C0218E1C6
:101AE000C12ED12C00E4402E83E1A82E82E0B82E36
:101AF00090E1592E80919502853009F044C012E1A1
:101B000080919502853009F038C08091950284302B
:101B100021F180E00E94ED1A109280020FB6F89435
:101B2000A895C09260000FBE4092600083B7817F8D
:101B3000846083BF83B7816083BF7894889583B7BF
:101B40008E7F83BF0FB6F894A8958091600088615E
:101B500080936000109260000FBE809194028823F1
:101B600009F4CECF0E949F13E9E0F2E08191811148
:101B70007DC1AE16BF06D1F7C3CF0E94D4240E9408
:101B8000DA1B0E94531A0E949F1381110E94BF19F1
:101B9000A9E0B2E0E4E1F2E000E010E0802E9D90E8
:101BA0008191892549F1E12CFF24F3949F2D9823FD
:101BB000F1F00E941711882399F0E9828A829F2010
:101BC00081E009F480E08B830E94CB198160782F3B
:101BD0009D838C8349815A816B818D810E941F0373
:101BE000F801EC5EFD4F8081F826F0821AC0E39484
:101BF000FF0C96E0E912DACF0F5F1F4F0A30110594
:101C000069F68FEF8E838F8318860E94CB198160CF
:101C1000782F9A8789874E815F8168858A850E949F
:101C20001F030E94171180914802882309F4BDC048
:101C300080914702E0917102E695E81BE093430230
:101C4000823059F4F0E0EA51FF4FE4910E2F10E09A
:101C5000B1E9EB2EB8E1FB2E59C0863059F4F0E023
:101C6000ED51FF4FE4910E2F10E0A1E8EA2EA8E11C
:101C7000FA2E4CC0893061F4E695F0E0E052FF4F57
:101C8000E4910E2F10E0F6E0EF2EF8E1FF2E3EC0BB
:101C90008F3061F4E695F0E0E352FF4FE4910E2FB0
:101CA00010E0EAE6EE2EE7E1FE2E30C0853159F471
:101CB000F0E0E652FF4FE4910E2F10E074EEE72EB5
:101CC00076E1F72E23C08831A1F0833249F4E8EDA4
:101CD000F0E00591149161E4E62E68E1F62E16C05D
:101CE000843271F404EF11E052E1E52E56E1F52E55
:101CF0000DC008E210E041E5E42E46E1F42E06C0F6
:101D000000ED17E03EEAE32E35E1F32E8091440228
:101D1000882361F0109244020E946C119093420259
:101D20008093410210924602109245020E946C116B
:101D3000E0914102F09142029C012E1B3F0B2F3F8C
:101D40003F4798F5209120022223B1F01092200203
:101D500020911E0230911F02821B930B8F3F9F47E1
:101D600058F4205D3A4830931F0220931E02809160
:101D70004902886080934902809045029090460213
:101D80000E0F1F1F109342020093410281E492E064
:101D9000F70109958091450290914602892B29F41B
:101DA000892819F081E08093200280912502E82F94
:101DB000EE0FEE0FE093250283B185FB662460F8F9
:101DC000712C93B1892F90E0880F892F881F990B70
:101DD000009711F082E090E0862997298E2B80935E
:101DE0002502109124028F70E82FF0E0EA59FE4F8F
:101DF000908180912302890F8093230284306CF0BC
:101E0000E12FF0E0EF5DFD4F80818F5F808360E028
:101E1000812F0E94C70321E001C020E080912302AE
:101E20008D3F64F4E12FF0E0EF5DFD4F8081815044
:101E3000808361E0812F0E94C70321E0809123020B
:101E4000082E000C990B64E070E00E94EC2A80934D
:101E5000230221110E94FE120E94531A9091260221
:101E6000891709F447CE8093260244CE59BC19BD88
:101E700009B400FEFDCF8091D8008F7D8093D800FB
:101E80008091E00082608093E0008091E00081FD1D
:101E9000FCCF0E94D42434CEAF92BF92CF92DF9277
:101EA000EF92FF920F931F93CF93DF937C015B011F
:101EB0006A018091F4018A3018F001E010E002C05C
:101EC0000AE010E0C1E0D0E0F894B501C701F601E6
:101ED00009957894811115C021960C171D0794F06F
:101EE000CC9F9001CD9F300D300D112480E090E00B
:101EF00045E34A95F1F70000019682179307C1F771
:101F0000E3CF81E0DF91CF911F910F91FF90EF9090
:101F1000DF90CF90BF90AF90089580E008959091AA
:101F2000050292FF0DC0282F2871283019F4877FF1
:101F3000846006C0282F2471243011F48B7F8860C0
:101F400093FF0DC0282F2871283119F4877E8461F2
:101F500006C0282F2471243111F48B7E88612091D2
:101F6000060220FF0DC0382F3871383019F4877FF2
:101F7000816006C0382F3171313011F48E7F886056
:101F800021FF0DC0282F2871283119F4877E816127
:101F900006C0282F2171213111F48E7E886194FDB5
:101FA000877E08958F929F92AF92BF92CF92DF92D9
:101FB000EF92FF920F931F93CF93DF93FB018080EB
:101FC0009180A280B3809FB7F894C0908102D09096
:101FD0008202E0908302F09084029FBFC818D90863
:101FE000EA08FB08F4E6CF16D104E104F10410F48A
:101FF000442341F17B01C82F880FDD0B011511052A
:10200000A9F0FE0183E0EE0FFF1F8A95E1F7E05093
:10201000FF4F818192818D529E4F408150E0041785
:10202000150708F4A801B9010E947F2BCE010E9478
:10203000F729882341F00E94BF19F701608371835B
:102040008283938381E0DF91CF911F910F91FF9065
:10205000EF90DF90CF90BF90AF909F908F900895BA
:102060006F927F928F929F92AF92BF92CF92DF92A8
:10207000EF92FF920F931F93CF93DF931F92CDB7F1
:10208000DEB7C62E4A015901682E880F7708C301B2
:102090000E94F729882309F473C0C30123E0880F45
:1020A000991F2A95E1F7FC01E050FF4F438150E072
:1020B0004115510511F041E050E0FC01E050FF4FA7
:1020C000648175816D527E4FCE0101960E947F2BF7
:1020D000F40140815181628173812FB7F89480911E
:1020E000810290918202A0918302B09184022FBF5D
:1020F000841B950BA60BB70B84369105A105B10582
:1021000038F4B701C8010E94D61A99818917D1F114
:102110000C2C000CDD08C6010E94F729782E8823BC
:10212000E1F0E114F104C9F0960183E0220F331FBE
:102130008A95E1F7F901E050FF4F438150E0E41642
:10214000F50608F4A701F901E050FF4F648175819D
:102150006D527E4FC5010E947F2BB701C8010E94BE
:10216000D61A91E02981281390E0D92ED72089F042
:102170000E94BF19F401608371838283938309C035
:10218000D12C02C0DD24D394A701B801C5010E945F
:102190007F2B8D2D0F90DF91CF911F910F91FF908D
:1021A000EF90DF90CF90BF90AF909F908F907F90F7
:1021B0006F900895CF92DF92EF92FF920F931F934B
:1021C000CF93DF9300D000D01F92CDB7DEB76B0165
:1021D00085E0E82EF12C04ED11E09E012F5F3F4FCA
:1021E0004DE352E061E080E00E943010882349F026
:1021F00095E0FE013196A8E3B2E001900D929A9528
:10220000E1F795E0E8E3F2E0D60101900D929A95AE
:10221000E1F70F900F900F900F900F90DF91CF91FB
:102220001F910F91FF90EF90DF90CF9008958091D4
:102230003702811118C08091D80080618093D80046
:102240008AE18A95F1F700C08091D90080FD02C033
:1022500082E001C081E080933702823021F40E9445
:102260009C1F1092950281E090913702913009F005
:1022700080E00895F894E82FE295EF70F0E031A146
:10228000282F2F7081E090E001C0880F2A95EAF78F
:10229000982F9095932391A392A1892B82A3789450
:1022A00008950F931F930E941711882321F01F9107
:1022B0000F910C94BF190E94BF190091F501109164
:1022C000F6012091F7013091F801600F711F821F14
:1022D000931F1F910F9108950E94171181110C9463
:1022E000CB190E945111CB010895CF93DF9382380F
:1022F000910569F1B0F48133910509F46FC048F498
:102300008932910509F465C08A32910509F46BC0E0
:102310008AC08533910509F457C089339105B9F016
:1023200082C0833E910571F138F4803E9105B1F091
:10233000823E910511F177C0863E9105B9F1873E45
:102340009105C9F1843E910509F06DC024C020912A
:10235000050220FD53C021FD51C065C080910502DA
:1023600080FD46C08091060280FF48C08091050232
:1023700084FD3FC183EE90E03EC18091050282FF63
:102380003AC0F4CF8091050282FD35C080910602EB
:1023900080FD34C0EBCF8091060281FF35C0809173
:1023A000050284FD26C187EE90E025C180910502DB
:1023B00083FF27C0F4CF8091050283FD22C0809166
:1023C000060281FD21C0EBCF8091050285FD1FC073
:1023D00021C08091050285FD1DC019C080910502B4
:1023E00086FD1BC01DC08091050286FD19C015C069
:1023F00089E390E000C182EE90E0FDC080EE90E0C5
:10240000FAC086EE90E0F7C084EE90E0F4C089E276
:1024100090E0F1C085E390E0EEC08AE290E0EBC08E
:1024200081E390E0E8C0811532E5930708F069C0C8
:10243000811541E5940728F0982F8827816F906ACD
:10244000DAC0883E910568F5803E910508F0D3C05A
:10245000883A9105B8F4853A910548F0855AE82FF5
:10246000F0E0EA58FE4F808190E09064C4C0813073
:10247000910509F4BBC008F4BCC08430910508F490
:10248000B8C0B9C08F3B910508F0B3C0885AE82F97
:10249000F0E0EE0FFF1FE758FE4F808191819464BA
:1024A000AAC0811520E59207F0F09C0174E03695F2
:1024B00027957A95E1F7922F9370482F437021E08A
:1024C00030E002C0220F331F4A95E2F73C68392BF7
:1024D0008F70982F9695969540E2949FC001112495
:1024E000822B932B88C0811530E4930718F09F70DE
:1024F000906A81C09C013A9521153F4108F47BC048
:1025000078C0EC01C11586E5D807E8F5C11525E5C9
:10251000D20748F08C2F0E948F0F8F7190E0982F78
:102520008827906268C0C11534E5D30728F09C2F36
:102530008827846F906A5FC0AE01437055272C2FA7
:1025400026952695C115D34578F481E090E002C028
:10255000880F991F4A95E2F740E2249F90011124C9
:10256000822B932B9C6847C081E090E002C0880FCB
:10257000991F4A95E2F740E2249F90011124822B93
:10258000932B9A6838C0C1152AE5D207F8F4C11513
:1025900039E5D30790F08C2F8F700E948F0F94E055
:1025A000D695C7959A95E1F7CF70D0E0DC2FCC2770
:1025B000D0699E01282BC9011EC0C11548E5D4076A
:1025C000C0F09C2F8827806F906A15C0CE0190566E
:1025D0008115904270F48D2F8F710E948F0F282FDC
:1025E0002F71CE0199279062922B05C081E090E077
:1025F00002C080E090E0DF91CF9108950C94BF1964
:10260000CF9384E090E00E94722AC82F82E290E08B
:102610000E94722A2C2F30E0A901582BCA01CF91B9
:10262000089569EE7EEF80E090E00E94A42A60E0C9
:1026300082E090E00E94862A60E083E090E00E94C1
:10264000862A1092290210922A0210922B021092CE
:102650002C0260E084E090E00E94862A60E082E242
:1026600090E00E94862A60E085E090E00E94862A41
:1026700060E086E090E00E94862A6FEF87E090E0BD
:102680000E94862A40E050E0BA0188E090E00E9473
:10269000982A60E08DE090E00E94862A40E050E0B9
:1026A000BA0188E190E00E94982A60E087E190E01A
:1026B0000E94862A40E050E0BA018CE190E00E943E
:1026C000982A60E070E080E290E00E94A42A40E056
:1026D00050E0BA0188E190E00E94982A0E94C21B53
:1026E00083E00E94A51BE1E7F2E0808181608083A6
:1026F00086950E94A72721E04FEF6FEF80E00E94B0
:1027000083268BE00E94A72740E050E0BA018FE0CB
:1027100090E00E94982A40E050E0BA0183E190E006
:102720000C94982A80912802811110922802089511
:1027300080959091270289238093270208955F92C4
:102740006F927F928F929F92AF92BF92CF92DF92C1
:10275000EF92FF920F931F93CF93DF93CDB7DEB726
:102760002F970FB6F894DEBF0FBECDBF9E012F5F2F
:102770003F4F79018AE0D9011D928A95E9F70BE56F
:1027800011E0690180E6682E81E0782EAA24A394E6
:10279000B12C26E6822E21E0922EF80180818F3F17
:1027A00009F440C0F894E82FE295EF70F0E021A121
:1027B0008F70A50102C0440F551F8A95E2F7CA0128
:1027C000922F982B91A392A18095892382A378942C
:1027D00000C0E0E6F1E0512C31E021912F3F89F07B
:1027E000A22FA295AF70B0E090968C9190E02F70E0
:1027F00002C0959587952A95E2F780FD02C0832F48
:1028000001C080E0582A330F8E169F0631F7D80199
:102810008C918F3F11F00E943A11B0EABA95F1F70E
:10282000F60150820F5F1F4FFFEFCF1ADF0A6016CD
:10283000710609F0B2CF4AE050E0B70189EF91E0AC
:102840000E94722B8C01892B41F08AE0F701A9EFDD
:10285000B1E001900D928A95E1F7F0900402011524
:10286000110549F081E080932F020E94CB199093CB
:102870002E0280932D0280912F028823B9F080913F
:102880002D0290912E020E94B019059778F0A9EFC1
:10289000B1E0EF2DF0E0E75FFD4F8EEF91E02D917D
:1028A00021938A179B07D9F710922F020115110562
:1028B00009F026C10E941711E09104029E01255FD4
:1028C0003F4F7901882309F46DC085E0D9011D923D
:1028D0008A95E9F70E2F10E0075F1D4F8091F401F4
:1028E0008A3048F44AED50E1B701C8010E944C0F0C
:1028F000882359F10AC080913002909131020E94E0
:10290000B019843F914070F732C044EC5BE0B701EE
:10291000C8010E944C0F8823C1F04CE65BE0B70170
:10292000C8010E944C0F882381F045E45BE0B701A9
:10293000C8010E944C0F882341F04AE05BE0B701D8
:10294000C8010E944C0F8111DEC08091F4018F3FBD
:1029500019F08F5F8093F4018091F4018A3008F4BC
:10296000D4C00E94CB1990933102809330028091A1
:102970003602811102C000E0D9C085E0F701119252
:102980008A95E9F710923602A0910302B0E0A75FA2
:10299000BD4F85E0FE013B9601900D928A95E1F7CF
:1029A00001E0C4C0F0E0E75FFD4FF89485E0A4EDDE
:1029B000B1E001900D928A95E1F765E070E084ED59
:1029C00091E00E94D61A8093D3017894F894E09114
:1029D0002402F0E0EF5DFD4F80818B878093DA0168
:1029E00061E070E0C7010E94D61A8093D901789403
:1029F000F894C090DB01D090DC01E090DD01F09014
:102A0000DE018091320290913302A0913402B091A4
:102A10003502C816D906EA06FB06D1F0C09232028A
:102A2000D0923302E0923402F09235020E941711E4
:102A300081110EC00E94BF19C61AD70AE80AF90A06
:102A4000C092F501D092F601E092F701F092F80100
:102A50007894F8948091DF010E94ED1A7894F894AC
:102A60008091E701882309F449C080FF24C0909138
:102A7000E0018091710290FF09C081608093710232
:102A800060E0892F86950E94672715C08E7F80930E
:102A900071020E941F1C809149028160809349024B
:102AA000FFEF20E732E0F15020403040E1F700C076
:102AB00000000E940E258091E70181FF09C020E0FF
:102AC0004091E3016091E2018091E1010E9483263F
:102AD0008091E70182FF09C08091E601882319F007
:102AE0000E94261C02C00E941F1C8091E70183FFE8
:102AF00003C081E0809344021092E701789416C0ED
:102B000001E010E013C01092F4018091030290E004
:102B100045E050E0B701875F9D4F0E94722B21E096
:102B200020933602892B09F02FCF25CF802F2F96A7
:102B30000FB6F894DEBF0FBECDBFDF91CF911F91CE
:102B40000F91FF90EF90DF90CF90BF90AF909F904C
:102B50008F907F906F905F900895089508950895E5
:102B600080918A0208958093850270938702609312
:102B7000860280919502843001F582E08093E9001D
:102B80008FEF9091E800815095FD06C095ED9A95E4
:102B9000F1F700008111F5CF8091E80085FF0DC0AD
:102BA00040E050E063E070E085E892E00E945F1C46
:102BB0008091E8008E778093E8000895BC0184E05E
:102BC0000C94B315BC0183E00C94B315CF93DF9341
:102BD00021E02093E9002FEF3091E800215035FDEE
:102BE00006C035ED3A95F1F700002111F5CF20919F
:102BF000E80025FF14C0EC0140E050E068E070E020
:102C00000E945F1C8091E8008E778093E80088E046
:102C1000FE01ABE8B2E001900D928A95E1F7DF91F9
:102C2000CF9108950F931F93CF93DF93EC0100E0B2
:102C300010E080915701282F30E00217130724F588
:102C4000909155019801290F311DA901440F551F7D
:102C5000240F351F235B3D4F869590E04C8108176C
:102C600019071CF4442331F002C0411103C0409104
:102C7000740201C040E060917302809172020E9470
:102C8000D3250F5F1F4FD5CF0E940E258C8190E07A
:102C90000196817099278C83DF91CF911F910F91BD
:102CA00008958F929F92AF92BF92CF92DF92EF9250
:102CB000FF920F931F93CF93DF938C01FC0144810C
:102CC000C42FD0E09E01DE010E94302B9B01AC019D
:102CD0000E94462B6B017C01E0E2F0E0EC1BFD0B57
:102CE000A5E5B0E09B01AC010E94462B4B015C01C5
:102CF0009F01DF010E94282B9B01AC010E94512BF8
:102D00009B01AC012C0D3D1D4E1D5F1DC501B40185
:102D10000E94002BC22FD22F2A3228F4F3E02F9FDB
:102D2000900111240DC025E530E02C1B3109C901AB
:102D3000880F991F280F391F37FF02C02F5F3F4FA1
:102D400035952795C22FC095F12C85E5E82EED1A13
:102D500080915701F816C8F4F1FC02C08E2D01C015
:102D60008D2F909155012F2D30E0290F311DA90194
:102D7000440F551F240F351F235B3D4F4C2F60918F
:102D800073020E94D325F394E3CF0E940E25F8012D
:102D90008481811102C091E003C0803219F49FEF59
:102DA0009093520190915201890FF8018483DF9131
:102DB000CF911F910F91FF90EF90DF90CF90BF9038
:102DC000AF909F908F9008951F93CF93DF93EC0166
:102DD0008C81811109C081E08C8310924B0292E0BA
:102DE000909351018093500180915501909156012B
:102DF000891770F4E82FF0E09F01220F331FE20FD4
:102E0000F31FE35BFD4F1182108212828F5FF0CFC0
:102E100010E0609157011617C0F5E12FF0E070E067
:102E2000CF010E94EC2A20915501820F20914B0284
:102E3000022E000C330B90E0E217F307CCF0209148
:102E40005101022E000C330B2E173F078CF09C0112
:102E5000220F331F820F931F9C01235B3D4F409134
:102E6000740260917302809172020E94D3250BC09C
:102E7000FC01EE0FFF1F8E0F9F1FFC01E35BFD4F58
:102E80001182108212821F5FC4CF0E940E25809192
:102E9000500120914B02280F20934B029091510139
:102EA000980F9093510119165CF4022E000C330B0D
:102EB0004091570150E0415051092417350734F033
:102EC000819580935001813009F41C82DF91CF916C
:102ED0001F9108957F928F929F92AF92BF92CF924F
:102EE000DF92EF92FF920F931F93CF93DF93EC014A
:102EF0008A8180FF03C0BB24BA9402C0BB24B39470
:102F00008C8181110DC081E0B81206C080915701FB
:102F1000815080934A0202C010924A0281E08C8361
:102F2000A12C4CE0842E90905701A91408F041C0C8
:102F300080915501CA2CD12C8601080F111DC801A2
:102F4000880F991F080F191F035B1D4FF80111828D
:102F50001082128234E0E32EF12C712C80914A020F
:102F6000870D8D302CF0682D0E94CA2A892F02C04F
:102F700087FD890D082E000C990BC816D90691F40F
:102F8000809174028E9DA0018F9D500D1124559546
:102F9000479555954795980160917302809172020B
:102FA0000E94D3257B0CF1E0EF1AF108B9F6A39447
:102FB000BACF0E940E2580914A0291E0B9120EC04C
:102FC000811107C080915701815080934A021C8271
:102FD0000FC0815080934A02BC820AC090E00196E3
:102FE0006091570170E00E94EC2A80934A028C8322
:102FF000DF91CF911F910F91FF90EF90DF90CF90D5
:10300000BF90AF909F908F907F900895FF920F9305
:103010001F93CF93DF93EC01F12C0FEF10E0609141
:103020005701F616F0F4809155012F2D30E0280F4E
:10303000311DC901880F991F280F391F235B3D4F90
:1030400070E0C8010E94EC2A962F8C814091740296
:1030500060917302F99E800D11240E94D325F39490
:10306000DECF0E940E259A818C8190FF02C08F5F77
:1030700001C081508C83DF91CF911F910F91FF9000
:1030800008950F931F93CF93DF9300D01F92CDB776
:10309000DEB78C0180914C0281110AC09E012F5F26
:1030A0003F4F4FEF6FEF0E94D3258A8180934C02F0
:1030B000F8018481813051F028F0823061F4409130
:1030C0004C020AC080914C0240E007C060914C0263
:1030D00040E080E003C040E080E060E00E945A25CC
:1030E000F801848190E0019663E070E00E94EC2A90
:1030F00084830F900F900F90DF91CF911F910F91CC
:103100000895CF93DF93EC01E1E7F2E04381628120
:103110008C810E9469268C818F5F8C83DF91CF9197
:103120000895CF93DF93EC01EC81F0E0E651FF4F7F
:103130004491E1E7F2E0628181810E9469268C81FD
:103140008F5F8C83DF91CF9108952091E4003091BF
:10315000E50095E64091EC00842F817040FF23C08C
:103160008091E80080FD1DC080919502882399F030
:10317000853099F08091EB0085FD11C04091E4000D
:103180005091E5002417350729F3915011F09A0169
:10319000E1CF84E0089582E0089583E0089581E01E
:1031A000089580E008954091E80042FFDDCF089542
:1031B0008091970287FF11C08091E80082FD05C0D1
:1031C000809195028111F8CF11C08091E8008B7732
:1031D0000BC080919502882349F08091E80080FF20
:1031E000F8CF8091E8008E778093E8000895982FBB
:1031F000973068F59093E900981739F07091EC00DA
:103200002091ED005091F00003C0242F762F50E064
:1032100021FD02C09F5FECCF3091EB003E7F3093E9
:10322000EB003091ED003D7F3093ED003091EB00ED
:1032300031603093EB007093EC002093ED005093DD
:10324000F0002091EE0027FDE5CF80E008958F701B
:103250008093E90081E0089520919D0230919E02C3
:103260002617370748F06115710539F42091E800F9
:103270002E772093E80001C0B901FC0120E0611520
:10328000710579F1809195028823F1F18530F1F192
:103290008091E80083FD3CC08091E80082FD2EC053
:1032A0008091E80080FFEBCF2091F3008091F20045
:1032B00090E0922B6115710551F08830910538F43A
:1032C00021912093F100615071090196F3CF21E023
:1032D000089709F020E08091E8008E778093E8005D
:1032E000CECF2111CFCF0AC080919502882361F003
:1032F000853061F08091E80083FD0AC08091E8008C
:1033000082FFF2CF80E0089582E0089583E008957F
:1033100081E0089578941F920F920FB60F921124B6
:103320008F939F93AF93BF9380918102909182027C
:10333000A0918302B09184020196A11DB11D8093DA
:10334000810290938202A0938302B0938402BF9182
:10335000AF919F918F910F900FBE0F901F90189576
:103360009C014FB7F8948091810290918202A091C4
:103370008302B09184024FBF821B930B08952FB735
:10338000F894609181027091820280918302909101
:1033900084022FBF08952FB7F894809181029091F5
:1033A0008202A0918302B09184022FBF08951F92E0
:1033B0000F920FB60F9211248F939F93AF93BF93E9
:1033C00080918002811113C08091810290918202CC
:1033D000A0918302B09184024196A11DB11D8093FA
:1033E000810290938202A0938302B0938402BF91E2
:1033F000AF919F918F910F900FBE0F901F901895D6
:103400009C012A5F3F4FFC014281461301C012829A
:10341000019682179307B9F708959C01FC01329633
:103420009FEF80E04191461789F09F3F19F44111C9
:1034300001C0982F8F5F8630A9F79F3F39F0F901BF
:10344000E90FF11D97FDFA95628308950895209183
:103450007E0230917F022817390771F090937F0226
:1034600080937E02E0917C02F0917D02309721F002
:103470000084F185E02D0994089520917A0230911D
:103480007B022817390771F090937B0280937A02B0
:10349000E0917C02F0917D02309721F00680F78167
:1034A000E02D099408950E941711882351F0E091AE
:1034B0007C02F0917D02309721F00190F081E02DA7
:1034C000099480E008950F931F93CF93DF93C42F47
:1034D000D22FFC0182818823C9F0409379020E9497
:1034E000CB19909378028093770280E28C0F88301A
:1034F00008F057C0C77081E001C0880FCA95EAF78D
:10350000DF91CF911F910F910C94E6248091790265
:10351000481330C080917702909178020E94B019D0
:10352000883C910538F510E21D0FCD17B9F080E207
:103530008C0F883040F4C77081E001C0880FCA95B5
:10354000EAF70E94DF24183028F581E09D2F97705C
:1035500001C0880F9A95EAF70E94E624802F0E9406
:10356000F0241830F0F4D77081E001C0880FDA95AC
:10357000EAF70AC080E28C0F883098F4C77081E0C7
:1035800001C0880FCA95EAF7DF91CF911F910F9183
:103590000C94DF24802FDF91CF911F910F910C9419
:1035A000F024DF91CF911F910F910895FC01680FD6
:1035B000791F8FEF91E3E617F70771F021918227CA
:1035C00028E030E087FF03C0880F892701C0880FFB
:1035D00021503109B9F7EFCF08958F929F92AF92A2
:1035E000BF92CF92DF92EF92FF920F931F93CF93F0
:1035F000DF93863048F4811108C0909180009F7D50
:10360000909380002E9806C085E090918000906293
:1036100090938000A0918600B0918700282F30E021
:103620000E94302B25E030E040E050E00E94002B6B
:103630000027122F232F342F012F122F232F332750
:1036400080918600909187006CE070E00E94D82AFB
:103650006017710730F0C80169E070E00E94D82A55
:103660005EC08091860090918700E0908600F09087
:103670008700E0918600F0918700C6E0D0E0BE01AF
:103680000E94D82A060F171F211D311D480159011C
:1036900085E0880C991CAA1CBB1C8A95D1F7C70130
:1036A000BE010E94D82A6F01E12CF12CA7019601DE
:1036B000260F371F411D511DC501B4010E94002B6B
:1036C00069017A01E0918600F0918700CA01B90191
:1036D0000E94BA2A9B01AC01DF010E94462B9B018C
:1036E000AC01C701B6010E94BA2ADC01CB012FE070
:1036F000B695A795979587952A95D1F7009186005D
:103700001091870020E030E0081719072A073B07CF
:1037100028F46091860070918700CB01BC01709302
:103720008B0060938A00DF91CF911F910F91FF90E2
:10373000EF90DF90CF90BF90AF909F908F900895C3
:10374000682F86E090E00C94862A863008F085E0A9
:10375000909176029770282F220F220F220F922B22
:1037600090937602987F21E009F420E09091760210
:1037700020FB90F9909376020E94ED1A80917602D8
:103780000C94A01B8091760280FD13C08160809311
:103790007602813019F489E0809376028091760276
:1037A0000E94A01B809176028695869586950C9442
:1037B000ED1A089580E090E00E94802A893E9E4F95
:1037C00051F00E9411138091760284708962809377
:1037D00076020E94A01B86E090E00E94722A8093ED
:1037E0007602282F26952695269530E0263031053D
:1037F00024F087708862809376028091760280FF41
:1038000004C086958695869501C080E00C94ED1ADB
:103810009091710290FF04C09695981740F003C0F4
:10382000811105C090E0961710F40C94B3270C9406
:10383000A727882311F0FA0101C0FB010994E7E4EE
:10384000F2E0118282818460828308956091710226
:10385000669570E04BE050E085E491E00E94652BB6
:10386000892B19F481E0809348020E946C11909397
:103870004202809341028091490284608093490210
:1038800008950F931F9380919F029091A002A091A1
:10389000A102B091A2028C019D010670112722277E
:1038A0003327BC01CD01063011052105310511F486
:1038B000686001C0677F1F910F910C944024EF92C4
:1038C000FF920F931F93CF93DF937C018B010E9494
:1038D000A518811119C0E70101151105A1F080910A
:1038E000E80085FD0AC08091E8008E778093E800AB
:1038F0000E94A518882381F307C089918093F10065
:1039000001501109E9CF80E0DF91CF911F910F9114
:10391000FF90EF9008951F93CF93DF93CDB7DEB75D
:10392000AA970FB6F894DEBF0FBECDBFE7E9F2E06D
:103930008FE992E02091F10021938E179F07D1F734
:1039400080919802833009F461C030F4813071F0C5
:10395000823009F49BC0B2C08A3009F487C08B3032
:1039600009F46CC0893009F0A9C020C08091970289
:10397000813A09F0A3C08091E800877F8093E80036
:1039800080919B0290919C02892B21F468E08BE846
:1039900092E003C060E080E090E070E00E942C19AB
:1039A0008091E8008B778093E80088C0809197022F
:1039B000813209F083C080919B0290919C02029712
:1039C00008F07CC08091E800877F8093E8008091B8
:1039D000E80082FD05C0809195028111F8CF6EC08C
:1039E0002091F3008091F20090E0922B029731F445
:1039F0008091F100813011F0863021F48091F10046
:103A000080938A028091E8008B7754C0809197025E
:103A1000813A09F053C080919B0290919C02892BBE
:103A200009F04CC08091E800877F8093E800809186
:103A3000E80080FFFCCF8091580137C08091970249
:103A40008132E1F580919B0290919C02892BB1F526
:103A50008091E800877F8093E8000E94D8188091C9
:103A60009902809358010E94D42428C08091970223
:103A7000813221F58091E800877F8093E8000E94E1
:103A8000D81880919A028093890218C08091970279
:103A9000813AA1F48091E800877F8093E8008091CB
:103AA000E80080FFFCCF809189028093F100809133
:103AB000E8008E778093E8000E94D8188091E80093
:103AC00083FFCEC18091970290919802492F50E0D8
:103AD0004A30510508F0C4C1FA01EE59FF4F0C9469
:103AE000222B803821F0823809F0BAC108C08091B9
:103AF000930290919402992389F082600FC0809183
:103B00009B028F70873008F0ABC18093E9008091F1
:103B1000EB0085FB882780F91092E9009091E8007E
:103B2000977F9093E8008093F1001092F10065C1B7
:103B3000282F2D7F09F094C1882319F0823061F07D
:103B40008FC180919902813009F08AC1933009F0C8
:103B500080E0809394022EC08091990281112AC046
:103B600080919B028F702FEF280F263008F078C1CC
:103B70008093E9002091EB0020FF1CC0933021F4DA
:103B80008091EB00806214C09091EB009061909363
:103B9000EB0021E030E0A90102C0440F551F8A95D7
:103BA000E2F74093EA001092EA008091EB0088600F
:103BB0008093EB001092E9008091E800877F20C19C
:103BC00081114EC1109199021F778091E300807896
:103BD000812B8093E3008091E800877F8093E80049
:103BE0000E94D8188091E80080FFFCCF8091E3000C
:103BF00080688093E300111102C082E001C083E07D
:103C0000809395022DC18058823008F029C180919F
:103C1000990290919A028C3D53E0950779F583E0E3
:103C20008A838AE289834FB7F894DE01139620E0F5
:103C30003EE051E2E32FF0E050935700E49120FF83
:103C400003C0E295EF703F5FEF708E2F90E0EA3097
:103C500010F0C79601C0C0968D939D932F5F2431BD
:103C600049F74FBF8091E800877F8093E8006AE2C0
:103C700070E0CE0101960E942C19AEC040919B02CB
:103C800050919C02292F332723303105A9F068F485
:103C90002130310509F4F3C02230310509F0E0C0CC
:103CA0008BE390E0ECE5F2E044C02132310521F1F4
:103CB0002232310571F1D4C0992781309105A1F0EC
:103CC00058F0029709F0CCC0E9EAF2E0E4918E2FB7
:103CD00090E0E9EAF2E02AC0E1EEF2E0E4918E2F12
:103CE00090E0E1EEF2E022C0E1EDF2E0E4918E2F0F
:103CF00090E0E1EDF2E01AC04115510509F4C4C0AD
:103D00004130510509F0ACC089E090E0E7E8F2E00D
:103D100010C04115510509F4BCC04130510509F0EE
:103D20009FC082E390E0EAEEF1E003C0009709F45F
:103D300097C02091E800277F2093E80020919D0202
:103D400030919E028217930708F49C0140E02115F0
:103D5000310589F180919502882309F43DC08530B1
:103D6000D9F18091E80083FD37C08091E80082FDA1
:103D70002FC08091E80080FFEACF4091F30080914E
:103D8000F20090E0942B2115310559F0883091050F
:103D900040F444914093F10031962150310901964D
:103DA000F2CF41E0089709F040E08091E8008E777B
:103DB0008093E800CCCF4111CDCF0AC0809195020D
:103DC000882351F0853041F08091E80083FD04C0E4
:103DD0008091E80082FFF2CF8091E8008B7780939A
:103DE000E8003EC08038E1F58091E800877F80934D
:103DF000E800809196028093F1008091E8008E7730
:103E00008093E8000E94D8182BC0811129C08091AE
:103E1000990290919A029927029714F58091E800EF
:103E2000877F8093E80010919902109396020E9478
:103E3000D818111106C08091E30087FD02C081E00F
:103E400001C084E08093950242E061EC81E00E9431
:103E5000F71842E261EC82E00E94F7188091950227
:103E60008091E80083FF1AC08091E800877F8093EB
:103E7000E8008091EB0080628093EB000FC082E14C
:103E800090E0E7E9F2E055CF89E090E0EEE6F2E07D
:103E900050CF80E490E0ECE1F2E04BCFAA960FB671
:103EA000F894DEBF0FBECDBFDF91CF911F91089573
:103EB0001F920F920FB60F9211242F933F934F939F
:103EC0005F936F937F938F939F93AF93BF93CF93A2
:103ED000DF93EF93FF93C091E900CF708091EC00E6
:103EE000D82FD17080FDD0E81092E9008091F000C9
:103EF000877F8093F00078940E948B1C1092E900D9
:103F00008091F00088608093F000CD2BCF70C0933B
:103F1000E900FF91EF91DF91CF91BF91AF919F9118
:103F20008F917F916F915F914F913F912F910F9062
:103F30000FBE0F901F901895E8EDF0E080818E7F06
:103F400080831092E2001092DA001092E100A0EE5D
:103F5000B0E08C9181608C9380818F77808319BCD5
:103F6000A7EDB0E08C918E7F8C9380818F7E8083D3
:103F7000109288020895CF92DF92EF92FF920F93F2
:103F80001F93CF93DF93C8EDD0E088818F7E888325
:103F9000E7EDF0E080818160808384E082BF81E092
:103FA0008093880288818E7F888302EE10E0F8017A
:103FB00010821092DA0081EEC82ED12CF601108208
:103FC00088818F77888388818068888388818F7DC6
:103FD000888319BC10929502109296021092940256
:103FE0001092930290EEE92EF12CF70180818B7FE5
:103FF000808388818160888342E060E080E00E9465
:10400000F718F60180818E7F8083F80180818160BE
:104010008083808188608083F70180818E7F8083A8
:10402000888180618883DF91CF911F910F91FF90EC
:10403000EF90DF90CF9008951F920F920FB60F92DE
:1040400011242F933F934F935F936F937F938F939D
:104050009F93AF93BF93EF93FF938091E10082FF13
:1040600009C08091E20082FF05C08091E1008B7F52
:104070008093E1008091DA0080FF2AC08091D8000F
:1040800080FF26C08091DA008E7F8093DA008091D5
:10409000D90080FF18C080E189BD82E189BD09B4E3
:1040A00000FEFDCF81E0809395028091880281110E
:1040B0000FC00E949C1F0E94BB1F8091E200846081
:1040C0008093E20005C019BC1092950210928802FC
:1040D0008091E10080FF17C08091E20080FF13C053
:1040E0008091E2008E7F8093E2008091E200806107
:1040F0008093E2008091D80080628093D80019BC40
:1041000085E0809395028091E10084FF30C080912A
:10411000E20084FF2CC080E189BD82E189BD09B441
:1041200000FEFDCF8091D8008F7D8093D8008091D4
:10413000E1008F7E8093E1008091E2008F7E80938A
:10414000E2008091E20081608093E200809196021B
:10415000882311F084E007C08091E30087FD02C04E
:1041600081E001C083E08093950280919502809167
:10417000E10083FF27C08091E20083FF23C080918C
:10418000E100877F8093E10082E0809395021092A6
:1041900096028091E1008E7F8093E1008091E200A1
:1041A0008E7F8093E2008091E20080618093E20044
:1041B00042E060E080E00E94F7188091F0008860A3
:1041C0008093F000FF91EF91BF91AF919F918F91FC
:1041D0007F916F915F914F913F912F910F900FBE03
:1041E0000F901F9018959091270280911403982B9F
:1041F0009093A30280912802882389F0892B8093D1
:10420000A302E5EAF2E097E080E0915029F02191E5
:104210002223D9F38F5FF9CF81110E94921348E0D6
:1042200050E06CE073E083EA92E00E94722B892BED
:10423000A9F088E0E3EAF2E0ACE0B3E001900D928F
:104240008A95E1F7E0917C02F0917D02309731F0A0
:104250000280F381E02D83EA92E00994089580E0E2
:1042600090E00E943D1A80E090E00E94271A109290
:1042700014030C94F32080910A039091D9028917BA
:1042800019F08F5F8770FBCF08950F931F93CF9323
:10429000DF938091D80282958F7009F05DC0809184
:1042A000D502882309F458C080910A031091D902DD
:1042B0006091D3027091D402C091D602D091D702FE
:1042C00091E06F3F09F090E0292F06E0811709F493
:1042D00043C0209721F07F3F21F030E003C031E060
:1042E00001C0322F90E030FD34C0089FF001099FDB
:1042F000F00D1124DF01A652BD4F11963C9111978C
:10430000371327C03C91361324C012963C91129764
:1043100031111FC013964D915C9114974C1B5D0B8E
:10432000483C5105B0F48091D8028F708061809331
:10433000D802E152FD4F80818F708061808383EDD0
:1043400092E00E94DA03DF91CF911F910F910C94BC
:104350003B2101968770BACFDF91CF911F910F91CA
:1043600008958F929F92AF92BF92DF92EF92FF9249
:104370000F931F93CF93DF9380909F029090A002A2
:10438000A090A102B090A2024091290250912A026D
:1043900060912B0270912C02842A952AA62AB72AB2
:1043A000CFE1D0E026E0929F700111249CE3D92E4A
:1043B000082F10E0D501C4010C2E04C0B695A795B6
:1043C000979587950A94D2F780FD04C0219790F7BE
:1043D00080E014C0DC9EF001DD9EF00D1124EE0D96
:1043E000FF1DE00FF11FEE0FFF1FEB51FD4F8591F9
:1043F00094910E947511019749F38C2FDF91CF9111
:104400001F910F91FF90EF90DF90BF90AF909F9022
:104410008F900895CF93DF93EC010E94B1212CE39C
:10442000829FC0011124FC0126E0D29FE00DF11D06
:104430001124EC0FF11DEE0FFF1FEB51FD4F859185
:1044400094910E947511DF91CF910895FC018081B4
:1044500091810E940A2292959F70963079F010F413
:10446000925001C09A50923068F4803F69F018F47D
:10447000883E40F409C0843F29F406C0883E20F0FD
:10448000813F11F080E0089581E008959F92AF92FE
:10449000BF92CF92DF92EF92FF920F931F93CF9331
:1044A000DF93CDB7DEB761970FB6F894DEBF0FBECE
:1044B000CDBF8C0185E0F801DE011D9601900D92C3
:1044C0008A95E1F7F801E2809091D3026091D402DD
:1044D0004091D6025091D7024115510531F06F3FFE
:1044E00031F481E09F3F19F403C081E001C080E016
:1044F000F82FF1709F2E80FD1AC1F80130812181C3
:10450000C380D48083EDA82E82E0B82EF090D5022F
:10451000F601E41BF50BFF2009F4C6C08091D80218
:10452000E83CF10508F091C0482F407F09F050C0E9
:10453000621311C093130FC0FE2CE1100CC08F70DA
:1045400080618093D802C5010E94DA038091D8026D
:10455000F801858329C1CD2831F02F3F31F481E066
:104560003F3F19F403C081E001C080E080FD03C03B
:1045700081E08E2502C080E090E0F82FF170FF2EE0
:1045800080FF1CC080910A034091D90256E0841735
:1045900009F4E8C090E0589FF001599FF00D1124F4
:1045A000E652FD4F6181261306C06081631303C08C
:1045B0006281E61203C001968770E9CFFE2CEE20DF
:1045C00009F4F2C08091D80281608093D80249C07A
:1045D000621306C0931304C0E11002C0F80186C044
:1045E000C8010E942622882351F1EE2041F120913A
:1045F000D802822F82958F7090E0029774F080919C
:10460000D3029091D40298878F831986DB86CA865D
:104610002C87CE0107960E94DA0386E0F801A3ED0D
:10462000B2E001900D928A95E1F70E9445210AC0FF
:104630006217C9F0C8010E94262281111EC0C8015C
:104640000E94DA03FF24F394AFC0482F407F81F724
:1046500083ED92E00E94DA0386E0F50111928A95DB
:10466000E9F7F12CA1C09313E5CFE110E3CFF801F6
:104670008583C8010E94DA0354C0EE2001F3209123
:10468000D802822F82958F7090E0029734F2809149
:10469000D3029091D4029A8389831B82DD82CC82DB
:1046A0002E83CE010196B7CFE83CF105D0F5FE2C64
:1046B000EE2029F2621327C0931325C02091D8025F
:1046C00020FD18C0822F82958F70482F50E0411531
:1046D000510581F0F80125834F30510541F08F5F7E
:1046E000982F9295907F822F8F70892B8583C80198
:1046F0000E94DA0386E0F801A3EDB2E001900D928A
:104700008A95E1F751C0C8010E942622811185CF08
:104710008091D80281608093D802C8010E94DA0398
:1047200043C086E0F50111928A95E9F73DC0EE207D
:1047300009F485CFC8010E942622F82E882309F4A7
:104740007ECF86E0F801A3EDB2E001900D928A954C
:10475000E1F78091D3029091D4020E940A220E9434
:10476000452122C03D872E878D859E850E940A2285
:10477000292F22952F70223028F49F7039F0811153
:1047800005C00BC0243028F49F7049F4805E883047
:1047900020F0C8010E94DA039F2CF92C05C0F80113
:1047A0009581907F99F7F9CF8F2D61960FB6F89488
:1047B000DEBF0FBECDBFDF91CF911F910F91FF9054
:1047C000EF90DF90CF90BF90AF909F900895292FEA
:1047D000220F920F990F890F682F6695669566953F
:1047E000982F977085E0689FB001112440E050E059
:1047F00080E0FB01E40FF51FE555FD4F208130E01F
:10480000092E02C0369527950A94E2F721703327C6
:10481000042E01C0220F0A94EAF7822B4F5F5F4FEC
:104820004530510531F70895292F220F920F990F26
:10483000890FE82FE695E695E695877051E001C06F
:10484000550F8A95EAF785E0E89FF0011124E555B8
:10485000FD4F20E030E070E04081CB01022E02C02D
:10486000969587950A94E2F7817081958427852330
:10487000842781932F5F3F4F2530310569F70895D5
:1048800060939F027093A0028093A1029093A20272
:104890000C942F210F931F9341E050E060E070E0F3
:1048A00004C0440F551F661F771F8A95D2F74095A5
:1048B00050956095709580919F029091A002A09173
:1048C000A102B091A2028A019B01082319232A2385
:1048D0003B23C901B8011F910F910C9440242091F2
:1048E0000B038095822380930B03982F977099F484
:1048F00030E0482F082E000C550B2417350759F0CF
:104900009091060292FD07C08595859585950E9438
:104910004A2410920B030895CF93C0910602C2FB64
:10492000992790F9981799F080FBC2F9C093060275
:104930006091050284E090E00E94862A6C2F82E25A
:1049400090E00E94862A82E0CF910C946F24CF9150
:1049500008950F931F9341E050E060E070E004C0C1
:10496000440F551F661F771F8A95D2F780919F02CB
:104970009091A002A091A102B091A2028A019B0194
:10498000082B192B2A2B3B2BC901B8011F910F9122
:104990000C9440246093290270932A0280932B0286
:1049A00090932C020C942F211092270286E0E5EAC6
:1049B000F2E0DF011D928A95E9F70C942F218823FC
:1049C00021F00E9498130C94F3200895882339F065
:1049D00090912702892B809327020C94F32008954D
:1049E0001F93CF93DF93182F893319F0C0E0D0E0E5
:1049F00002C0C0E5D0E0812F0E941428209741F02A
:104A00008FE99FE00197F1F700C000002197F6CFF2
:104A1000812FDF91CF911F910C94BD2730915401CC
:104A20008091710280FF16C0E091530163E0E69F20
:104A3000F0011124E35BFD4F879A81B38F7791B327
:104A400090682FB7F894AF0163E0369F400D511D79
:104A5000112414C08091550190915601891720F7B7
:104A6000E82FF0E0AF01440F551FE40FF51FE35BA3
:104A7000FD4F1182108212828F5FF0CFE417F5078D
:104A800089F0319168E091BB000000C037FF81BB25
:104A9000330F000000C000C000C081BB00C06A9599
:104AA00091F7ECCF2FBF8FE594E00197F1F700C0AD
:104AB000000008959091710290FF16C090915501E9
:104AC00020915601921770F4E92FF0E0DF01AA0F50
:104AD000BB1FEA0FFB1FE35BFD4F818360834283B3
:104AE0009F5FF0CF0C940E25089580917102282FBE
:104AF000269530E02115310519F48170826005C0DA
:104B00002532310524F08170886480937102089504
:104B1000CF92DF92EF92FF926B017C010E9475258C
:104B2000B701A60188E090E0FF90EF90DF90CF9072
:104B30000C94982A80917502882319F081508093F3
:104B4000750260917102709172028091730290916E
:104B500074020C94882580917502833018F48F5F5D
:104B6000809375026091710270917202809173025C
:104B7000909174020C948825E1E7F2E083E0808351
:104B800011828FEF828383831482A7E4B2E01296AE
:104B90008C911297836012968C93608171818281CF
:104BA00093810C948825AF92BF92CF92DF92EF92BF
:104BB000FF920F931F93CF93DF93E82EF62EE90118
:104BC000E42FF0E0611106C0EB53FB4FE4914E2F50
:104BD0002E2F71C0062F10E0EB53FB4F4491F42FA2
:104BE000C42ED12C26E0829FC00111242FEF30E08B
:104BF000B9010E94D82A5BEA5603C001579F900D65
:104C000011248E0D911D8E0D911D582F550F580F8B
:104C1000D901A01BB10BAC9DC001AD9D900DBC9DF9
:104C2000900D1124E92FF59ED0011124AB2FBB2745
:104C30007901EA1AFB0AEC9CD001ED9CB00DFC9CBA
:104C4000B00D11245901A51AB108A09E7001A19EB2
:104C5000F00CB09EF00C1124EF2CFF242E193F090C
:104C60002C9D80012D9D100D3C9D100D1124212F98
:104C70006230710591F048F461157105E1F0613021
:104C80007105B9F4242F4B2F16C06430710569F0FB
:104C900040F06630710579F00CC0242F492FE12FC8
:104CA0000AC0492FEF2F2B2F06C0292FE42F412FA9
:104CB00002C0292FEB2F49832883EA83DF91CF910C
:104CC0001F910F91FF90EF90DF90CF90BF90AF902A
:104CD0000895CF93DF9300D01F92CDB7DEB79091A8
:104CE000710290FF0AC09E012F5F3F4F0E94D325A3
:104CF0004B8169818A810E945A250F900F900F90F5
:104D0000DF91CF910895AF92BF92CF92DF92EF9251
:104D1000FF920F931F93CF93DF9300D01F92CDB7D5
:104D2000DEB7182FF62E042FE22E9091710290FF1D
:104D30007EC0E92FE695AE2FB0E0A955BE4F8C910D
:104D4000809347029E7F923061F49E012F5F3F4F18
:104D5000812F0E94D3254B8169818A810E945A2527
:104D600043C0823019F4009174023EC0863019F4B9
:104D70001091720239C08930D9F38931A9F5E9510E
:104D80008E2F8170D82EE695F0E0EB53FA4FA59068
:104D9000B490C12CBB2460915701C61618F52C2D78
:104DA00030E0A29EC001A39E900DB29E900D1124F2
:104DB00070E00E94D82A812FD11002C0860F01C056
:104DC000861B90915501290F311DA901440F551FD4
:104DD000240F351F235B3D4F402F6F2D0E94D3259D
:104DE000C394D9CF0E940E2580917202181308C077
:104DF00080917302F81204C080917402081729F0A0
:104E00008091490282608093490210937202F0926D
:104E1000730200937402EE2051F060917102709160
:104E2000720280917302909174020E9488250F9003
:104E30000F900F90DF91CF911F910F91FF90EF9006
:104E4000DF90CF90BF90AF900895E1E7F2E043810B
:104E500021E1421B08F440E021E0628181810C9451
:104E60008326E1E7F2E0438121E1420F08F44FEFAE
:104E700021E0628181810C948326E1E7F2E0628186
:104E800021E1621B08F460E021E0438181810C9400
:104E90008326E1E7F2E0628121E1620F08F46FEF1F
:104EA00021E0438181810C948326E1E7F2E0818156
:104EB00021E04381628188500C948326E1E7F2E08F
:104EC000818121E043816281885F0C9483269091E7
:104ED000710290FF3BC09170811102C0926006C0C8
:104EE000853210F0986402C0880F982B909371025D
:104EF00080914902816080934902662351F060915C
:104F000071027091720280917302909174020E94FA
:104F1000882560917102669570E04BE050E085E471
:104F200091E00E94652B892B19F00E941F1C02C082
:104F30000E94261C81E08093440220E0409174028C
:104F400060917302809172020C948326089561E04F
:104F50000C946727809171028695815009F484E250
:104F600061E00C9467278091710286958F5F85328E
:104F700008F081E061E00C946727882309F453C0AE
:104F8000682F823869F40E94531A81FF4CC069E38C
:104F900083EA92E00E940D1A0E94F32069E30EC09A
:104FA000833891F40E94531A80FF3DC063E583EA81
:104FB00092E00E940D1A0E94F32063E583EA92E0DA
:104FC0000E94001A0C94F320843869F40E94531A4A
:104FD00082FF29C067E483EA92E00E940D1A0E94D2
:104FE000F32067E4EBCF8CEF860F813A38F380E251
:104FF000860F883048F4677081E001C0880F6A9599
:10500000EAF70E949813DECF8BE5860F833020F4F9
:1050100080E090E00C943D1A685A673120F480E0FB
:1050200090E00C94271A0895CF93882309F496C032
:10503000C82F8238B1F40E94531A81FD8FC069E3F2
:1050400083EA92E00E940D1A0E94F3202FEF81EE76
:1050500094E0215080409040E1F700C0000069E3F7
:1050600017C08338E1F40E94531A80FD77C063E5CE
:1050700083EA92E00E940D1A0E94F3202FEF81EE46
:1050800094E0215080409040E1F700C0000063E5CB
:1050900083EA92E00E94001ACF910C94F3208438A6
:1050A000B1F40E94531A82FD59C067E483EA92E08A
:1050B0000E940D1A0E94F3202FEF81EE94E0215000
:1050C00080409040E1F700C0000067E4E1CF8CEF42
:1050D0008C0F813A80F4E5EAF2E08BEA92E02191CC
:1050E000C217A1F18E179F07D1F76C2F83EA92E0C8
:1050F0000E940D1AD1CF80E28C0F883068F4C770FF
:1051000081E090E001C0880FCA95EAF790912702EC
:10511000892B80932702C0CFEBE5EC0FE33040F4FE
:10512000F0E0EA58FE4F808190E0CF910C943D1A58
:10513000C85AC73198F4EC2FF0E0EE0FFF1FE75884
:10514000FE4F80819181CF910C94271A6C2F83EAB6
:1051500092E00E94001A0E94F320C7CFCF910895D9
:105160008EE1489B02C08150E1F7489BFECF089535
:10517000589880E28A95F1F7589A0895FC012AE040
:105180002A95F1F728E090E080E031E040E14A958F
:10519000F1F7880F489B02C08160932700C0000090
:1051A00040E14A95F1F7215089F720E12A95F1F77E
:1051B00029B100C0000030E13A95F1F72170922743
:1051C0002081920F90830895EF92FF920F931F9387
:1051D000CF93DF931F92CDB7DEB719828C017C018C
:1051E000E60EF11C0E151F0551F00E94B028CE01ED
:1051F00001960E94BE28F80181938F01F3CF81E0D0
:105200009981911180E00F90DF91CF911F910F91C3
:10521000FF90EF900895509A589A08955098589A90
:10522000E89AE9E6F0E080818C7F80830895615000
:1052300091E001C0990F6A95EAF720E031E09923E7
:1052400061F0492F482319F0589A232701C0589834
:1052500040E24A95F1F79695F2CF222311F0589A41
:1052600001C0589880E28A95F1F758980895FF9206
:105270000F931F93CF93DF93EC018C01060F111D49
:10528000C017D10741F0F9900E94B82868E08F2D2F
:105290000E941729F5CFDF91CF911F910F91FF90B9
:1052A00008951F920F920FB60F9211240F931F9320
:1052B0002F933F934F935F936F937F938F939F931E
:1052C000AF93BF93EF93FF93CF93DF931F92CDB72D
:1052D000DEB719820E94B028CE0101960E94BE2836
:1052E000082F069506950695902F96959570202F78
:1052F0002570920F292F237096959695920F87709F
:1053000089135FC0898181115CC0083008F059C0E1
:1053100080E18A95F1F7589A509A82E08A95F1F7E0
:1053200000C0589888E0089F80011124D801A0503F
:10533000BF4F1696ED91FC9117973097A9F06091A9
:10534000590170915A0114962D913C911597260F91
:10535000371F11968D919C911297680F791F1396A4
:105360004C9113978C910995F801E050FF4F6381A0
:10537000662351F08091590190915A012481358121
:10538000820F931F0E9437290E94B82880E18A95D6
:10539000F1F758985098589A80E18A95F1F7F801FA
:1053A000E050FF4F6081662351F080915901909148
:1053B0005A0121813281820F931F0E94E4280E94AA
:1053C000B0280F90DF91CF91FF91EF91BF91AF91F6
:1053D0009F918F917F916F915F914F913F912F910D
:1053E0001F910F910F900FBE0F901F9018950F9364
:1053F0001F93CF93DF93883091050CF06DC0EC01C3
:10540000F894509A589885E08A95F1F700009C2FFF
:10541000969595702C2F2570920F892F83709695F5
:10542000969523E0CC0FDD1F2A95E1F7980F8E01AA
:10543000092B0E94B82884E08A95F1F700C068E043
:10544000802F0E94172980E18A95F1F75098589A89
:10545000489902C000C0FCCF87E090E0489B08C09C
:10546000019721F4509A589A789436C000C0F6CF2C
:10547000FE01E050FF4F6381662381F08091590166
:1054800090915A0124813581820F931F0E94E42854
:10549000811104C0509A589A78941FC00E94B02875
:1054A00080E28A95F1F75898509A80E18A95F1F751
:1054B000C050DF4F6881662351F08091590190916F
:1054C0005A0129813A81820F931F0E9437290E9435
:1054D000B828789481E001C080E0DF91CF911F91DE
:1054E0000F910895F999FECF92BD81BDF89A992741
:1054F00080B50895A6E1B0E044E050E00C94AC2AF9
:10550000A8E1B0E042E050E00C94AC2A262FF999D3
:10551000FECF92BD81BDF89A019700B4021639F012
:105520001FBA20BD0FB6F894FA9AF99A0FBE0895E3
:105530000396272F0E94872A0E94862A252F0E94E1
:10554000872A242F0C94872A0196272F0E94872AC6
:105550000C94862ADC01CB01FC01F999FECF06C030
:10556000F2BDE1BDF89A319600B40D924150504021
:10557000B8F70895DB018F939F930E94462BBF914C
:10558000AF91A29F800D911DA39F900DB29F900D92
:105590001124089587FB082E062687FD819567FD57
:1055A00061950E94592B0EF4919507FC8195089501
:1055B000AA1BBB1B51E107C0AA1FBB1FA617B70739
:1055C00010F0A61BB70B881F991F5A95A9F7809555
:1055D0009095BC01CD01089597FB072E16F4009419
:1055E00007D077FD09D00E94D82A07FC05D03EF4E9
:1055F000909581959F4F0895709561957F4F08957F
:10560000A1E21A2EAA1BBB1BFD010DC0AA1FBB1FC6
:10561000EE1FFF1FA217B307E407F50720F0A21B38
:10562000B30BE40BF50B661F771F881F991F1A94A5
:1056300069F760957095809590959B01AC01BD01CF
:10564000CF010895EE0FFF1F0590F491E02D09940E
:105650000E94302B332312F48A1B9B0B0C94412B9A
:10566000A29FB001B39FC001A39F700D811D1124A3
:10567000911DB29F700D811D1124911D08950E94EE
:10568000302BB7FF0895821B930B08950E94302B97
:10569000A59F900DB49F900DA49F800D911D112486
:1056A0000895B7FF0C94462B0E94462B821B930B48
:1056B0000895991B79E004C0991F961708F0961B6E
:1056C000881F7A95C9F780950895FC014150504094
:1056D00030F001900616D1F73197CF010895882751
:1056E00099270895FB01DC0104C08D910190801978
:1056F00021F441505040C8F7881B990B0895FB01D5
:10570000DC0102C001900D9241505040D8F708953D
:04571000F894FFCF3B
:10571400000000010000000000000005010000007E
:105724000000000106000000000000010700000066
:105734000408000000000000010C0000000000004C
:10574400080D00000000000001B015E615AF15E2D9
:1057540015DE15AD1501191A1B1C1D1E1F20212253
:10576400010201000C000C0C01D301929395979651
:10577400F1F4F5F6943400FF0100010000FFFF008E
:1057840000010001FF00818283E200E900EA00B524
:1057940000B600B700CD008301CC008A01920194C9
:1057A400012102230224022502260227022A02B32F
:1057B40000B4006F00700000010202020206060637
:1057C4000909090909090F0F0F0F0F0F15151518EE
:0C57D40019191919191919191919232488
:00000001FF
